 isfldsin003

 Timestamp is a328e96e (reproducible build file hash)

 Preferred load address is 0000000180000000

 Start         Length     Name                   Class
 0001:00000000 00002bf0H .text$mn                CODE
 0001:00002bf0 00000036H .text$mn$00             CODE
 0001:00002c26 00000092H .text$x                 CODE
 0002:00000000 00000198H .idata$5                DATA
 0002:00000198 00000038H .00cfg                  DATA
 0002:000001d0 00000008H .CRT$XCA                DATA
 0002:000001d8 00000008H .CRT$XCZ                DATA
 0002:000001e0 00000008H .CRT$XIA                DATA
 0002:000001e8 00000008H .CRT$XIC                DATA
 0002:000001f0 00000008H .CRT$XIZ                DATA
 0002:000001f8 00000008H .CRT$XLA                DATA
 0002:00000200 00000008H .CRT$XLZ                DATA
 0002:00000208 00000008H .CRT$XPA                DATA
 0002:00000210 00000008H .CRT$XPZ                DATA
 0002:00000218 00000008H .CRT$XTA                DATA
 0002:00000220 00000010H .CRT$XTZ                DATA
 0002:00000228 00000000H .gehcont$y              DATA
 0002:00000228 00000000H .gfids$y                DATA
 0002:00000230 00001bd0H .rdata                  DATA
 0002:00001e00 00000000H .rdata$CastGuardVftablesA DATA
 0002:00001e00 00000000H .rdata$CastGuardVftablesC DATA
 0002:00001e00 00000028H .rdata$T                DATA
 0002:00001e28 000000a4H .rdata$voltmd           DATA
 0002:00001ecc 0000031cH .rdata$zzzdbg           DATA
 0002:000021e8 00000008H .rtc$IAA                DATA
 0002:000021f0 00000008H .rtc$IZZ                DATA
 0002:000021f8 00000008H .rtc$TAA                DATA
 0002:00002200 00000008H .rtc$TZZ                DATA
 0002:00002208 00000004H .tls                    DATA
 0002:0000220c 00000004H .tls$                   DATA
 0002:00002210 00000008H .tls$ZZZ                DATA
 0002:00002218 000002e8H .xdata                  DATA
 0002:00002500 000003a0H .edata                  DATA
 0002:000028a0 00000064H .idata$2                DATA
 0002:00002904 00000014H .idata$3                DATA
 0002:00002918 00000198H .idata$4                DATA
 0002:00002ab0 0000041eH .idata$6                DATA
 0003:00000000 000000b0H .data                   DATA
 0003:000000b0 0001b248H .bss                    DATA
 0004:00000000 00000378H .pdata                  DATA

  Address         Publics by Value              Rva+Base               Lib:Object

 0000:00000000       __AbsoluteZero             0000000000000000     <absolute>
 0000:00000000       ___safe_se_handler_count   0000000000000000     <absolute>
 0000:00000000       ___safe_se_handler_table   0000000000000000     <absolute>
 0000:00000000       __arm64x_extra_rfe_table   0000000000000000     <absolute>
 0000:00000000       __arm64x_extra_rfe_table_size 0000000000000000     <absolute>
 0000:00000000       __arm64x_native_entrypoint 0000000000000000     <absolute>
 0000:00000000       __arm64x_redirection_metadata 0000000000000000     <absolute>
 0000:00000000       __arm64x_redirection_metadata_count 0000000000000000     <absolute>
 0000:00000000       __dynamic_value_reloc_table 0000000000000000     <absolute>
 0000:00000000       __enclave_config           0000000000000000     <absolute>
 0000:00000000       __guard_check_icall_a64n_fptr 0000000000000000     <absolute>
 0000:00000000       __guard_eh_cont_count      0000000000000000     <absolute>
 0000:00000000       __guard_eh_cont_table      0000000000000000     <absolute>
 0000:00000000       __guard_fids_count         0000000000000000     <absolute>
 0000:00000000       __guard_fids_table         0000000000000000     <absolute>
 0000:00000000       __guard_iat_count          0000000000000000     <absolute>
 0000:00000000       __guard_iat_table          0000000000000000     <absolute>
 0000:00000000       __guard_longjmp_count      0000000000000000     <absolute>
 0000:00000000       __guard_longjmp_table      0000000000000000     <absolute>
 0000:00000000       __hybrid_auxiliary_iat     0000000000000000     <absolute>
 0000:00000000       __hybrid_auxiliary_iat_copy 0000000000000000     <absolute>
 0000:00000000       __hybrid_code_map          0000000000000000     <absolute>
 0000:00000000       __hybrid_code_map_count    0000000000000000     <absolute>
 0000:00000000       __x64_code_ranges_to_entry_points 0000000000000000     <absolute>
 0000:00000000       __x64_code_ranges_to_entry_points_count 0000000000000000     <absolute>
 0000:00000100       __guard_flags              0000000000000100     <absolute>
 0000:00000000       __ImageBase                0000000180000000     <linker-defined>
 0001:00000000       ?NewObject@JNIEnv_@@QEAAPEAV_jobject@@PEAV_jclass@@PEAU_jmethodID@@ZZ 0000000180001000 f i libisfldsin003.obj
 0001:00000028       ?TranslateError@@YAPEBDW4jvmtiError@@@Z 0000000180001028 f   libisfldsin003.obj
 0001:000002e0       ?nsk_jni_check_exception@@YAHPEAUJNIEnv_@@QEBDH@Z 00000001800012e0 f   libisfldsin003.obj
 0001:00000424       ?nsk_jni_lverify@@YAHHPEAUJNIEnv_@@HQEBDH1ZZ 0000000180001424 f   libisfldsin003.obj
 0001:000004c4       Agent_Initialize           00000001800014c4 f   libisfldsin003.obj
 0001:000005f8       Agent_OnAttach             00000001800015f8 f   libisfldsin003.obj
 0001:000005f8       Agent_OnLoad               00000001800015f8 f   libisfldsin003.obj
 0001:00000600       Java_nsk_jvmti_IsFieldSynthetic_isfldsin003a_check 0000000180001600 f   libisfldsin003.obj
 0001:00000788       Java_nsk_jvmti_unit_FollowReferences_FollowRefObjects_addRefToVerify 0000000180001788 f   libisfldsin003.obj
 0001:00000960       Java_nsk_jvmti_unit_FollowReferences_FollowRefObjects_getTag 0000000180001960 f   libisfldsin003.obj
 0001:00000a20       Java_nsk_jvmti_unit_FollowReferences_FollowRefObjects_resetRefsToVerify 0000000180001a20 f   libisfldsin003.obj
 0001:00000a28       Java_nsk_jvmti_unit_FollowReferences_FollowRefObjects_resetTags 0000000180001a28 f   libisfldsin003.obj
 0001:00000a6c       Java_nsk_jvmti_unit_FollowReferences_FollowRefObjects_setTag 0000000180001a6c f   libisfldsin003.obj
 0001:00000cc4       Java_nsk_share_jvmti_ArgumentHandler_getAgentOptionsString 0000000180001cc4 f   libisfldsin003.obj
 0001:00000d74       Java_nsk_share_jvmti_DebugeeClass_checkStatus 0000000180001d74 f   libisfldsin003.obj
 0001:00000dfc       Java_nsk_share_jvmti_DebugeeClass_resetAgentData 0000000180001dfc f   libisfldsin003.obj
 0001:00000e5c       Java_nsk_share_jvmti_RedefineAgent_agentStatus 0000000180001e5c f   libisfldsin003.obj
 0001:00000e68       Java_nsk_share_jvmti_RedefineAgent_isRedefined 0000000180001e68 f   libisfldsin003.obj
 0001:00000e74       Java_nsk_share_jvmti_RedefineAgent_redefineAttempted 0000000180001e74 f   libisfldsin003.obj
 0001:00000e80       MA_checkStatus             0000000180001e80 f   libisfldsin003.obj
 0001:00000f24       __local_stdio_printf_options 0000000180001f24 f i libisfldsin003.obj
 0001:00001104       exitOnError                0000000180002104 f   libisfldsin003.obj
 0001:000011b8       fprintf                    00000001800021b8 f i libisfldsin003.obj
 0001:000011fc       nsk_jvmti_lverify          00000001800021fc f   libisfldsin003.obj
 0001:000012ec       nsk_jvmti_resetAgentData   00000001800022ec f   libisfldsin003.obj
 0001:0000136c       nsk_jvmti_setFailStatus    000000018000236c f   libisfldsin003.obj
 0001:000013a8       nsk_lcomplain              00000001800023a8 f   libisfldsin003.obj
 0001:000013c8       nsk_ldisplay               00000001800023c8 f   libisfldsin003.obj
 0001:000013e8       nsk_ltrace                 00000001800023e8 f   libisfldsin003.obj
 0001:00001408       nsk_lvcomplain             0000000180002408 f   libisfldsin003.obj
 0001:000015c0       nsk_lvdisplay              00000001800025c0 f   libisfldsin003.obj
 0001:0000160c       nsk_lverify                000000018000260c f   libisfldsin003.obj
 0001:00001668       nsk_lvtrace                0000000180002668 f   libisfldsin003.obj
 0001:000016c8       nsk_printf                 00000001800026c8 f   libisfldsin003.obj
 0001:000016f0       nsk_vprintf                00000001800026f0 f   libisfldsin003.obj
 0001:000017a4       printf                     00000001800027a4 f i libisfldsin003.obj
 0001:00001ccc       __raise_securityfailure    0000000180002ccc f   MSVCRT:gs_report.obj
 0001:00001d00       __report_gsfailure         0000000180002d00 f   MSVCRT:gs_report.obj
 0001:00001f40       __GSHandlerCheck           0000000180002f40 f   MSVCRT:gshandler.obj
 0001:00001f60       __GSHandlerCheckCommon     0000000180002f60 f   MSVCRT:gshandler.obj
 0001:00001fd0       __security_check_cookie    0000000180002fd0 f   MSVCRT:amdsecgs.obj
 0001:00002310       _DllMainCRTStartup         0000000180003310 f   MSVCRT:dll_dllmain.obj
 0001:00002350       __scrt_acquire_startup_lock 0000000180003350 f   MSVCRT:utility.obj
 0001:0000238c       __scrt_dllmain_after_initialize_c 000000018000338c f   MSVCRT:utility.obj
 0001:000023c0       __scrt_dllmain_before_initialize_c 00000001800033c0 f   MSVCRT:utility.obj
 0001:000023d8       __scrt_dllmain_crt_thread_attach 00000001800033d8 f   MSVCRT:utility.obj
 0001:00002400       __scrt_dllmain_crt_thread_detach 0000000180003400 f   MSVCRT:utility.obj
 0001:00002418       __scrt_dllmain_exception_filter 0000000180003418 f   MSVCRT:utility.obj
 0001:00002478       __scrt_dllmain_uninitialize_c 0000000180003478 f   MSVCRT:utility.obj
 0001:000024a8       __scrt_dllmain_uninitialize_critical 00000001800034a8 f   MSVCRT:utility.obj
 0001:000024bc       __scrt_initialize_crt      00000001800034bc f   MSVCRT:utility.obj
 0001:00002508       __scrt_initialize_onexit_tables 0000000180003508 f   MSVCRT:utility.obj
 0001:00002594       __scrt_is_nonwritable_in_current_image 0000000180003594 f   MSVCRT:utility.obj
 0001:0000262c       __scrt_release_startup_lock 000000018000362c f   MSVCRT:utility.obj
 0001:00002650       __scrt_uninitialize_crt    0000000180003650 f   MSVCRT:utility.obj
 0001:0000267c       _onexit                    000000018000367c f   MSVCRT:utility.obj
 0001:000026b8       atexit                     00000001800036b8 f   MSVCRT:utility.obj
 0001:000026d0       __crt_debugger_hook        00000001800036d0 f   MSVCRT:utility_desktop.obj
 0001:000026d8       __scrt_fastfail            00000001800036d8 f   MSVCRT:utility_desktop.obj
 0001:00002824       _guard_check_icall_nop     0000000180003824 f i MSVCRT:guard_support.obj
 0001:00002828       __security_init_cookie     0000000180003828 f   MSVCRT:gs_support.obj
 0001:000028d4       DllMain                    00000001800038d4 f   MSVCRT:dll_dllmain_stub.obj
 0001:000028f8       ?__scrt_initialize_type_info@@YAXXZ 00000001800038f8 f   MSVCRT:tncleanup.obj
 0001:00002908       ?__scrt_uninitialize_type_info@@YAXXZ 0000000180003908 f   MSVCRT:tncleanup.obj
 0001:00002914       __local_stdio_scanf_options 0000000180003914 f i MSVCRT:default_local_stdio_options.obj
 0001:0000291c       __scrt_initialize_default_local_stdio_options 000000018000391c f   MSVCRT:default_local_stdio_options.obj
 0001:00002938       __scrt_get_dyn_tls_init_callback 0000000180003938 f   MSVCRT:dyn_tls_init.obj
 0001:00002940       _RTC_Initialize            0000000180003940 f   MSVCRT:initsect.obj
 0001:0000297c       _RTC_Terminate             000000018000397c f   MSVCRT:initsect.obj
 0001:000029b8       __isa_available_init       00000001800039b8 f   MSVCRT:cpu_disp.obj
 0001:00002b64       _get_startup_argv_mode     0000000180003b64 f   MSVCRT:argv_mode.obj
 0001:00002b6c       __scrt_is_ucrt_dll_in_use  0000000180003b6c f   MSVCRT:ucrt_detection.obj
 0001:00002b80       memcpy                     0000000180003b80 f   vcruntime:VCRUNTIME140.dll
 0001:00002b86       memset                     0000000180003b86 f   vcruntime:VCRUNTIME140.dll
 0001:00002b8c       strchr                     0000000180003b8c f   vcruntime:VCRUNTIME140.dll
 0001:00002b92       __C_specific_handler       0000000180003b92 f   vcruntime:VCRUNTIME140.dll
 0001:00002b98       __std_type_info_destroy_list 0000000180003b98 f   vcruntime:VCRUNTIME140.dll
 0001:00002b9e       strcmp                     0000000180003b9e f   ucrt:api-ms-win-crt-string-l1-1-0.dll
 0001:00002ba4       strlen                     0000000180003ba4 f   ucrt:api-ms-win-crt-string-l1-1-0.dll
 0001:00002baa       _initterm                  0000000180003baa f   ucrt:api-ms-win-crt-runtime-l1-1-0.dll
 0001:00002bb0       _initterm_e                0000000180003bb0 f   ucrt:api-ms-win-crt-runtime-l1-1-0.dll
 0001:00002bb6       _seh_filter_dll            0000000180003bb6 f   ucrt:api-ms-win-crt-runtime-l1-1-0.dll
 0001:00002bbc       _configure_narrow_argv     0000000180003bbc f   ucrt:api-ms-win-crt-runtime-l1-1-0.dll
 0001:00002bc2       _initialize_narrow_environment 0000000180003bc2 f   ucrt:api-ms-win-crt-runtime-l1-1-0.dll
 0001:00002bc8       _initialize_onexit_table   0000000180003bc8 f   ucrt:api-ms-win-crt-runtime-l1-1-0.dll
 0001:00002bce       _register_onexit_function  0000000180003bce f   ucrt:api-ms-win-crt-runtime-l1-1-0.dll
 0001:00002bd4       _execute_onexit_table      0000000180003bd4 f   ucrt:api-ms-win-crt-runtime-l1-1-0.dll
 0001:00002bda       _crt_atexit                0000000180003bda f   ucrt:api-ms-win-crt-runtime-l1-1-0.dll
 0001:00002be0       _cexit                     0000000180003be0 f   ucrt:api-ms-win-crt-runtime-l1-1-0.dll
 0001:00002be8       __acrt_initialize          0000000180003be8 f   MSVCRT:ucrt_stubs.obj
 0001:00002be8       __acrt_thread_attach       0000000180003be8 f   MSVCRT:ucrt_stubs.obj
 0001:00002be8       __acrt_thread_detach       0000000180003be8 f   MSVCRT:ucrt_stubs.obj
 0001:00002be8       __acrt_uninitialize        0000000180003be8 f   MSVCRT:ucrt_stubs.obj
 0001:00002be8       __acrt_uninitialize_critical 0000000180003be8 f   MSVCRT:ucrt_stubs.obj
 0001:00002be8       __scrt_stub_for_acrt_initialize 0000000180003be8 f   MSVCRT:ucrt_stubs.obj
 0001:00002be8       __scrt_stub_for_acrt_thread_attach 0000000180003be8 f   MSVCRT:ucrt_stubs.obj
 0001:00002be8       __scrt_stub_for_acrt_thread_detach 0000000180003be8 f   MSVCRT:ucrt_stubs.obj
 0001:00002be8       __scrt_stub_for_acrt_uninitialize 0000000180003be8 f   MSVCRT:ucrt_stubs.obj
 0001:00002be8       __scrt_stub_for_acrt_uninitialize_critical 0000000180003be8 f   MSVCRT:ucrt_stubs.obj
 0001:00002be8       __vcrt_initialize          0000000180003be8 f   MSVCRT:ucrt_stubs.obj
 0001:00002be8       __vcrt_thread_attach       0000000180003be8 f   MSVCRT:ucrt_stubs.obj
 0001:00002be8       __vcrt_thread_detach       0000000180003be8 f   MSVCRT:ucrt_stubs.obj
 0001:00002be8       __vcrt_uninitialize        0000000180003be8 f   MSVCRT:ucrt_stubs.obj
 0001:00002be8       __vcrt_uninitialize_critical 0000000180003be8 f   MSVCRT:ucrt_stubs.obj
 0001:00002bec       __scrt_stub_for_is_c_termination_complete 0000000180003bec f   MSVCRT:ucrt_stubs.obj
 0001:00002bec       _is_c_termination_complete 0000000180003bec f   MSVCRT:ucrt_stubs.obj
 0001:00002c00       _guard_dispatch_icall_nop  0000000180003c00 f   MSVCRT:guard_dispatch.obj
 0001:00002c20       _guard_xfg_dispatch_icall_nop 0000000180003c20 f   MSVCRT:guard_xfg_dispatch.obj
 0002:00000000       __imp_RtlCaptureContext    0000000180004000     kernel32:KERNEL32.dll
 0002:00000008       __imp_RtlLookupFunctionEntry 0000000180004008     kernel32:KERNEL32.dll
 0002:00000010       __imp_RtlVirtualUnwind     0000000180004010     kernel32:KERNEL32.dll
 0002:00000018       __imp_UnhandledExceptionFilter 0000000180004018     kernel32:KERNEL32.dll
 0002:00000020       __imp_SetUnhandledExceptionFilter 0000000180004020     kernel32:KERNEL32.dll
 0002:00000028       __imp_GetCurrentProcess    0000000180004028     kernel32:KERNEL32.dll
 0002:00000030       __imp_TerminateProcess     0000000180004030     kernel32:KERNEL32.dll
 0002:00000038       __imp_IsProcessorFeaturePresent 0000000180004038     kernel32:KERNEL32.dll
 0002:00000040       __imp_CloseHandle          0000000180004040     kernel32:KERNEL32.dll
 0002:00000048       __imp_InitializeCriticalSectionAndSpinCount 0000000180004048     kernel32:KERNEL32.dll
 0002:00000050       __imp_DeleteCriticalSection 0000000180004050     kernel32:KERNEL32.dll
 0002:00000058       __imp_CreateEventW         0000000180004058     kernel32:KERNEL32.dll
 0002:00000060       __imp_GetModuleHandleW     0000000180004060     kernel32:KERNEL32.dll
 0002:00000068       __imp_GetProcAddress       0000000180004068     kernel32:KERNEL32.dll
 0002:00000070       __imp_IsDebuggerPresent    0000000180004070     kernel32:KERNEL32.dll
 0002:00000078       __imp_QueryPerformanceCounter 0000000180004078     kernel32:KERNEL32.dll
 0002:00000080       __imp_GetCurrentProcessId  0000000180004080     kernel32:KERNEL32.dll
 0002:00000088       __imp_GetCurrentThreadId   0000000180004088     kernel32:KERNEL32.dll
 0002:00000090       __imp_GetSystemTimeAsFileTime 0000000180004090     kernel32:KERNEL32.dll
 0002:00000098       __imp_DisableThreadLibraryCalls 0000000180004098     kernel32:KERNEL32.dll
 0002:000000a0       __imp_InitializeSListHead  00000001800040a0     kernel32:KERNEL32.dll
 0002:000000a8       \177KERNEL32_NULL_THUNK_DATA 00000001800040a8     kernel32:KERNEL32.dll
 0002:000000b0       __imp_memcpy               00000001800040b0     vcruntime:VCRUNTIME140.dll
 0002:000000b8       __imp_memset               00000001800040b8     vcruntime:VCRUNTIME140.dll
 0002:000000c0       __imp_strchr               00000001800040c0     vcruntime:VCRUNTIME140.dll
 0002:000000c8       __imp___C_specific_handler 00000001800040c8     vcruntime:VCRUNTIME140.dll
 0002:000000d0       __imp___std_type_info_destroy_list 00000001800040d0     vcruntime:VCRUNTIME140.dll
 0002:000000d8       \177VCRUNTIME140_NULL_THUNK_DATA 00000001800040d8     vcruntime:VCRUNTIME140.dll
 0002:000000e0       __imp__errno               00000001800040e0     ucrt:api-ms-win-crt-runtime-l1-1-0.dll
 0002:000000e8       __imp_exit                 00000001800040e8     ucrt:api-ms-win-crt-runtime-l1-1-0.dll
 0002:000000f0       __imp__cexit               00000001800040f0     ucrt:api-ms-win-crt-runtime-l1-1-0.dll
 0002:000000f8       __imp__crt_atexit          00000001800040f8     ucrt:api-ms-win-crt-runtime-l1-1-0.dll
 0002:00000100       __imp__execute_onexit_table 0000000180004100     ucrt:api-ms-win-crt-runtime-l1-1-0.dll
 0002:00000108       __imp__register_onexit_function 0000000180004108     ucrt:api-ms-win-crt-runtime-l1-1-0.dll
 0002:00000110       __imp__initialize_onexit_table 0000000180004110     ucrt:api-ms-win-crt-runtime-l1-1-0.dll
 0002:00000118       __imp__initialize_narrow_environment 0000000180004118     ucrt:api-ms-win-crt-runtime-l1-1-0.dll
 0002:00000120       __imp__configure_narrow_argv 0000000180004120     ucrt:api-ms-win-crt-runtime-l1-1-0.dll
 0002:00000128       __imp__seh_filter_dll      0000000180004128     ucrt:api-ms-win-crt-runtime-l1-1-0.dll
 0002:00000130       __imp__initterm_e          0000000180004130     ucrt:api-ms-win-crt-runtime-l1-1-0.dll
 0002:00000138       __imp__initterm            0000000180004138     ucrt:api-ms-win-crt-runtime-l1-1-0.dll
 0002:00000140       \177api-ms-win-crt-runtime-l1-1-0_NULL_THUNK_DATA 0000000180004140     ucrt:api-ms-win-crt-runtime-l1-1-0.dll
 0002:00000148       __imp___acrt_iob_func      0000000180004148     ucrt:api-ms-win-crt-stdio-l1-1-0.dll
 0002:00000150       __imp_fflush               0000000180004150     ucrt:api-ms-win-crt-stdio-l1-1-0.dll
 0002:00000158       __imp___stdio_common_vsprintf 0000000180004158     ucrt:api-ms-win-crt-stdio-l1-1-0.dll
 0002:00000160       __imp___stdio_common_vfprintf 0000000180004160     ucrt:api-ms-win-crt-stdio-l1-1-0.dll
 0002:00000168       \177api-ms-win-crt-stdio-l1-1-0_NULL_THUNK_DATA 0000000180004168     ucrt:api-ms-win-crt-stdio-l1-1-0.dll
 0002:00000170       __imp_strcmp               0000000180004170     ucrt:api-ms-win-crt-string-l1-1-0.dll
 0002:00000178       __imp__strdup              0000000180004178     ucrt:api-ms-win-crt-string-l1-1-0.dll
 0002:00000178       __imp_strdup               0000000180004178     ucrt:api-ms-win-crt-string-l1-1-0.dll
 0002:00000180       __imp_strlen               0000000180004180     ucrt:api-ms-win-crt-string-l1-1-0.dll
 0002:00000188       __imp_strncpy              0000000180004188     ucrt:api-ms-win-crt-string-l1-1-0.dll
 0002:00000190       \177api-ms-win-crt-string-l1-1-0_NULL_THUNK_DATA 0000000180004190     ucrt:api-ms-win-crt-string-l1-1-0.dll
 0002:00000198       __guard_check_icall_fptr   0000000180004198     MSVCRT:guard_support.obj
 0002:000001a0       __guard_xfg_check_icall_fptr 00000001800041a0     MSVCRT:guard_support.obj
 0002:000001a8       __guard_dispatch_icall_fptr 00000001800041a8     MSVCRT:guard_support.obj
 0002:000001b0       __guard_xfg_dispatch_icall_fptr 00000001800041b0     MSVCRT:guard_support.obj
 0002:000001b8       __guard_xfg_table_dispatch_icall_fptr 00000001800041b8     MSVCRT:guard_support.obj
 0002:000001c0       __castguard_check_failure_os_handled_fptr 00000001800041c0     MSVCRT:guard_support.obj
 0002:000001c8       __guard_memcpy_fptr        00000001800041c8     vcruntime:softmemtag.obj
 0002:000001d0       __xc_a                     00000001800041d0     MSVCRT:initializers.obj
 0002:000001d8       __xc_z                     00000001800041d8     MSVCRT:initializers.obj
 0002:000001e0       __xi_a                     00000001800041e0     MSVCRT:initializers.obj
 0002:000001f0       __xi_z                     00000001800041f0     MSVCRT:initializers.obj
 0002:000001f8       __xl_a                     00000001800041f8     MSVCRT:tlssup.obj
 0002:00000200       __xl_z                     0000000180004200     MSVCRT:tlssup.obj
 0002:00000208       __xp_a                     0000000180004208     MSVCRT:initializers.obj
 0002:00000210       __xp_z                     0000000180004210     MSVCRT:initializers.obj
 0002:00000218       __xt_a                     0000000180004218     MSVCRT:initializers.obj
 0002:00000220       __xt_z                     0000000180004220     MSVCRT:initializers.obj
 0002:00000230       g_refKindStr               0000000180004230     libisfldsin003.obj
 0002:000003e0       ??_C@_09BPLDFGCI@unknown_0@ 00000001800043e0     libisfldsin003.obj
 0002:000003f0       ??_C@_0BL@FPNMECJD@JVMTI_HEAP_REFERENCE_CLASS@ 00000001800043f0     libisfldsin003.obj
 0002:00000410       ??_C@_0BL@FKGKKLNM@JVMTI_HEAP_REFERENCE_FIELD@ 0000000180004410     libisfldsin003.obj
 0002:00000430       ??_C@_0CD@CAEHCFJF@JVMTI_HEAP_REFERENCE_ARRAY_ELEM@ 0000000180004430     libisfldsin003.obj
 0002:00000458       ??_C@_0CC@DNEBMCNK@JVMTI_HEAP_REFERENCE_CLASS_LOAD@ 0000000180004458     libisfldsin003.obj
 0002:00000480       ??_C@_0BN@CJMIPEBB@JVMTI_HEAP_REFERENCE_SIGNERS@ 0000000180004480     libisfldsin003.obj
 0002:000004a0       ??_C@_0CH@HBOIDPEB@JVMTI_HEAP_REFERENCE_PROTECTION@ 00000001800044a0     libisfldsin003.obj
 0002:000004c8       ??_C@_0BP@MDKGDGKL@JVMTI_HEAP_REFERENCE_INTERFACE@ 00000001800044c8     libisfldsin003.obj
 0002:000004e8       ??_C@_0CC@JJMIHNJH@JVMTI_HEAP_REFERENCE_STATIC_FIE@ 00000001800044e8     libisfldsin003.obj
 0002:00000510       ??_C@_0CD@IDHEEGID@JVMTI_HEAP_REFERENCE_CONSTANT_P@ 0000000180004510     libisfldsin003.obj
 0002:00000538       ??_C@_0CA@EFFCHNG@JVMTI_HEAP_REFERENCE_SUPERCLASS@ 0000000180004538     libisfldsin003.obj
 0002:00000558       ??_C@_0L@PCDFHGCJ@unknown_11@ 0000000180004558     libisfldsin003.obj
 0002:00000568       ??_C@_0L@NJBICFOK@unknown_12@ 0000000180004568     libisfldsin003.obj
 0002:00000578       ??_C@_0L@MAADBEKL@unknown_13@ 0000000180004578     libisfldsin003.obj
 0002:00000588       ??_C@_0L@IPECICGM@unknown_14@ 0000000180004588     libisfldsin003.obj
 0002:00000598       ??_C@_0L@JGFJLDCN@unknown_15@ 0000000180004598     libisfldsin003.obj
 0002:000005a8       ??_C@_0L@LNHEOAOO@unknown_16@ 00000001800045a8     libisfldsin003.obj
 0002:000005b8       ??_C@_0L@KEGPNBKP@unknown_17@ 00000001800045b8     libisfldsin003.obj
 0002:000005c8       ??_C@_0L@CDPHMNGA@unknown_18@ 00000001800045c8     libisfldsin003.obj
 0002:000005d8       ??_C@_0L@DKOMPMCB@unknown_19@ 00000001800045d8     libisfldsin003.obj
 0002:000005e8       ??_C@_0L@OJGIPJDB@unknown_20@ 00000001800045e8     libisfldsin003.obj
 0002:000005f8       ??_C@_0CA@KAOFNDEM@JVMTI_HEAP_REFERENCE_JNI_GLOBAL@ 00000001800045f8     libisfldsin003.obj
 0002:00000618       ??_C@_0CC@HPFAJBK@JVMTI_HEAP_REFERENCE_SYSTEM_CLA@ 0000000180004618     libisfldsin003.obj
 0002:00000640       ??_C@_0BN@FDEGFOHC@JVMTI_HEAP_REFERENCE_MONITOR@ 0000000180004640     libisfldsin003.obj
 0002:00000660       ??_C@_0CB@HKIBCMAJ@JVMTI_HEAP_REFERENCE_STACK_LOCA@ 0000000180004660     libisfldsin003.obj
 0002:00000688       ??_C@_0BP@EAACMMOE@JVMTI_HEAP_REFERENCE_JNI_LOCAL@ 0000000180004688     libisfldsin003.obj
 0002:000006a8       ??_C@_0BM@IJDEOGOE@JVMTI_HEAP_REFERENCE_THREAD@ 00000001800046a8     libisfldsin003.obj
 0002:000006c8       ??_C@_0BL@EDGPPKC@JVMTI_HEAP_REFERENCE_OTHER@ 00000001800046c8     libisfldsin003.obj
 0002:000006e4       ??_C@_04BCJPDBDA@Code@     00000001800046e4     libisfldsin003.obj
 0002:000006f0       ??_C@_0BA@OCLMCFKC@LineNumberTable@ 00000001800046f0     libisfldsin003.obj
 0002:00000700       ??_C@_0BD@CPAEPILC@LocalVariableTable@ 0000000180004700     libisfldsin003.obj
 0002:00000718       ??_C@_0BH@NMBDNHBD@LocalVariableTypeTable@ 0000000180004718     libisfldsin003.obj
 0002:00000730       ??_C@_0O@HIHEEDNJ@StackMapTable@ 0000000180004730     libisfldsin003.obj
 0002:00000740       ??_C@_03IAKKBENL@fld@      0000000180004740     libisfldsin003.obj
 0002:00000744       ??_C@_01JPJNBJEM@I@        0000000180004744     libisfldsin003.obj
 0002:00000748       ??_C@_06JDLJJLAP@this$0@   0000000180004748     libisfldsin003.obj
 0002:00000750       ??_C@_0CK@HBNALOCL@Lnsk?1jvmti?1IsFieldSynthetic?1isf@ 0000000180004750     libisfldsin003.obj
 0002:00000780       ??_C@_0L@HCDIAMJG@?9?5?$CFs?0?5?$CFd?3?5@ 0000000180004780     libisfldsin003.obj
 0002:00000790       ??_C@_0JI@HLPECLFI@?$CD?5?4?4?4?6?$CD?5ERROR?3?5too?5many?5complai@ 0000000180004790     libisfldsin003.obj
 0002:00000830       ??_C@_0ED@JNEKCCOB@The?5following?5fake?5exception?5st@ 0000000180004830     libisfldsin003.obj
 0002:00000878       ??_C@_0CN@FCNMDFBH@nsk?4share?4Fake_Exception_for_RU@ 0000000180004878     libisfldsin003.obj
 0002:000008a8       ??_C@_08PGFFNAEI@?$CI?$CFs?3?$CFd?$CJ?5@ 00000001800048a8     libisfldsin003.obj
 0002:000008b8       ??_C@_0DP@IENMAEGI@s?2test?2hotspot?2jtreg?2vmTestbase@ 00000001800048b8     libisfldsin003.obj
 0002:000008f8       ??_C@_0BL@NDJLFFJB@?7at?5nsk_lvcomplain?$CI?$CFs?3?$CFd?$CJ?6@ 00000001800048f8     libisfldsin003.obj
 0002:00000918       ??_C@_0BC@JOOKAFKF@?$CD?5ERROR?3?5?$CFs?0?5?$CFd?3?5@ 0000000180004918     libisfldsin003.obj
 0002:00000930       ??_C@_09KJEAHMEH@?$CD?5ERROR?3?5@ 0000000180004930     libisfldsin003.obj
 0002:0000093c       ??_C@_02GPIOPFAK@?$DO?$DO@ 000000018000493c     libisfldsin003.obj
 0002:00000940       ??_C@_02FODMEDOG@?$DM?$DM@ 0000000180004940     libisfldsin003.obj
 0002:00000944       ??_C@_02DJGKEECL@?4?4@     0000000180004944     libisfldsin003.obj
 0002:00000948       ??_C@_0O@CJPGJOAF@?9?5?$CFs?0?5?$CFd?3?5?$CFs?5@ 0000000180004948     libisfldsin003.obj
 0002:00000958       ??_C@_0CB@IAKPDOIC@?$CD?5?5?5verified?5assertion?5is?5FALSE@ 0000000180004958     libisfldsin003.obj
 0002:00000980       ??_C@_0CO@LGONDEPD@stdout?3?5fflush?5failed?5?9?5err?$DN?$CFd?5@ 0000000180004980     libisfldsin003.obj
 0002:000009b0       ??_C@_0CO@KBGKJPBD@stderr?3?5fflush?5failed?5?9?5err?$DN?$CFd?5@ 00000001800049b0     libisfldsin003.obj
 0002:000009e0       ??_C@_0BB@JCNMKLLK@JVMTI_ERROR_NONE@ 00000001800049e0     libisfldsin003.obj
 0002:000009f8       ??_C@_0BL@LDIMKLPH@JVMTI_ERROR_INVALID_THREAD@ 00000001800049f8     libisfldsin003.obj
 0002:00000a18       ??_C@_0CB@PJFPAIKJ@JVMTI_ERROR_INVALID_THREAD_GROU@ 0000000180004a18     libisfldsin003.obj
 0002:00000a40       ??_C@_0BN@LLMKHMNF@JVMTI_ERROR_INVALID_PRIORITY@ 0000000180004a40     libisfldsin003.obj
 0002:00000a60       ??_C@_0CB@MBOFKAGB@JVMTI_ERROR_THREAD_NOT_SUSPENDE@ 0000000180004a60     libisfldsin003.obj
 0002:00000a88       ??_C@_0BN@FABOLPBI@JVMTI_ERROR_THREAD_SUSPENDED@ 0000000180004a88     libisfldsin003.obj
 0002:00000aa8       ??_C@_0BN@FDGNOBJM@JVMTI_ERROR_THREAD_NOT_ALIVE@ 0000000180004aa8     libisfldsin003.obj
 0002:00000ac8       ??_C@_0BL@GOBIFKNJ@JVMTI_ERROR_INVALID_OBJECT@ 0000000180004ac8     libisfldsin003.obj
 0002:00000ae8       ??_C@_0BK@FCMAJPPC@JVMTI_ERROR_INVALID_CLASS@ 0000000180004ae8     libisfldsin003.obj
 0002:00000b08       ??_C@_0BP@IKLLBKEB@JVMTI_ERROR_CLASS_NOT_PREPARED@ 0000000180004b08     libisfldsin003.obj
 0002:00000b28       ??_C@_0BN@KLPPLKG@JVMTI_ERROR_INVALID_METHODID@ 0000000180004b28     libisfldsin003.obj
 0002:00000b48       ??_C@_0BN@BCEKOKND@JVMTI_ERROR_INVALID_LOCATION@ 0000000180004b48     libisfldsin003.obj
 0002:00000b68       ??_C@_0BM@DFDGPME@JVMTI_ERROR_INVALID_FIELDID@ 0000000180004b68     libisfldsin003.obj
 0002:00000b88       ??_C@_0BL@NELIEPEC@JVMTI_ERROR_NO_MORE_FRAMES@ 0000000180004b88     libisfldsin003.obj
 0002:00000ba8       ??_C@_0BJ@BDBECFDM@JVMTI_ERROR_OPAQUE_FRAME@ 0000000180004ba8     libisfldsin003.obj
 0002:00000bc8       ??_C@_0BK@MIIFNLOB@JVMTI_ERROR_TYPE_MISMATCH@ 0000000180004bc8     libisfldsin003.obj
 0002:00000be8       ??_C@_0BJ@HPCAOILC@JVMTI_ERROR_INVALID_SLOT@ 0000000180004be8     libisfldsin003.obj
 0002:00000c08       ??_C@_0BG@CHILOPNI@JVMTI_ERROR_DUPLICATE@ 0000000180004c08     libisfldsin003.obj
 0002:00000c20       ??_C@_0BG@DIEMLHKM@JVMTI_ERROR_NOT_FOUND@ 0000000180004c20     libisfldsin003.obj
 0002:00000c38       ??_C@_0BM@NHMCKHOB@JVMTI_ERROR_INVALID_MONITOR@ 0000000180004c38     libisfldsin003.obj
 0002:00000c58       ??_C@_0BO@PPEDAJGL@JVMTI_ERROR_NOT_MONITOR_OWNER@ 0000000180004c58     libisfldsin003.obj
 0002:00000c78       ??_C@_0BG@FCAIPEID@JVMTI_ERROR_INTERRUPT@ 0000000180004c78     libisfldsin003.obj
 0002:00000c90       ??_C@_0CB@EGDBNKOI@JVMTI_ERROR_INVALID_CLASS_FORMA@ 0000000180004c90     libisfldsin003.obj
 0002:00000cb8       ??_C@_0CG@DGKOGIAL@JVMTI_ERROR_CIRCULAR_CLASS_DEFI@ 0000000180004cb8     libisfldsin003.obj
 0002:00000ce0       ??_C@_0BP@ICEALPKC@JVMTI_ERROR_FAILS_VERIFICATION@ 0000000180004ce0     libisfldsin003.obj
 0002:00000d00       ??_C@_0DC@JDACLMIO@JVMTI_ERROR_UNSUPPORTED_REDEFIN@ 0000000180004d00     libisfldsin003.obj
 0002:00000d38       ??_C@_0DE@GKDKNOMJ@JVMTI_ERROR_UNSUPPORTED_REDEFIN@ 0000000180004d38     libisfldsin003.obj
 0002:00000d70       ??_C@_0BO@LAFKIOG@JVMTI_ERROR_INVALID_TYPESTATE@ 0000000180004d70     libisfldsin003.obj
 0002:00000d90       ??_C@_0DH@INDGCLLB@JVMTI_ERROR_UNSUPPORTED_REDEFIN@ 0000000180004d90     libisfldsin003.obj
 0002:00000dc8       ??_C@_0DE@NHEOMMGI@JVMTI_ERROR_UNSUPPORTED_REDEFIN@ 0000000180004dc8     libisfldsin003.obj
 0002:00000e00       ??_C@_0CA@EKPNJOEP@JVMTI_ERROR_UNSUPPORTED_VERSION@ 0000000180004e00     libisfldsin003.obj
 0002:00000e20       ??_C@_0BN@OFFMAHHL@JVMTI_ERROR_NAMES_DONT_MATCH@ 0000000180004e20     libisfldsin003.obj
 0002:00000e40       ??_C@_0DN@HHBBLAKE@JVMTI_ERROR_UNSUPPORTED_REDEFIN@ 0000000180004e40     libisfldsin003.obj
 0002:00000e80       ??_C@_0DO@HMBGBGNA@JVMTI_ERROR_UNSUPPORTED_REDEFIN@ 0000000180004e80     libisfldsin003.obj
 0002:00000ec0       ??_C@_0BP@PBECGKHJ@JVMTI_ERROR_UNMODIFIABLE_CLASS@ 0000000180004ec0     libisfldsin003.obj
 0002:00000ee0       ??_C@_0BK@CANILEHF@JVMTI_ERROR_NOT_AVAILABLE@ 0000000180004ee0     libisfldsin003.obj
 0002:00000f00       ??_C@_0CE@INJKMEFK@JVMTI_ERROR_MUST_POSSESS_CAPABI@ 0000000180004f00     libisfldsin003.obj
 0002:00000f28       ??_C@_0BJ@LBFPFPDM@JVMTI_ERROR_NULL_POINTER@ 0000000180004f28     libisfldsin003.obj
 0002:00000f48       ??_C@_0BP@CHJPNNEM@JVMTI_ERROR_ABSENT_INFORMATION@ 0000000180004f48     libisfldsin003.obj
 0002:00000f68       ??_C@_0BP@OMFMNLC@JVMTI_ERROR_INVALID_EVENT_TYPE@ 0000000180004f68     libisfldsin003.obj
 0002:00000f88       ??_C@_0BN@BIBNPHHO@JVMTI_ERROR_ILLEGAL_ARGUMENT@ 0000000180004f88     libisfldsin003.obj
 0002:00000fa8       ??_C@_0BK@KKNDHDCE@JVMTI_ERROR_NATIVE_METHOD@ 0000000180004fa8     libisfldsin003.obj
 0002:00000fc8       ??_C@_0BK@PMKCFHAE@JVMTI_ERROR_OUT_OF_MEMORY@ 0000000180004fc8     libisfldsin003.obj
 0002:00000fe8       ??_C@_0BK@NNJBDMNB@JVMTI_ERROR_ACCESS_DENIED@ 0000000180004fe8     libisfldsin003.obj
 0002:00001008       ??_C@_0BI@GHECLMNC@JVMTI_ERROR_WRONG_PHASE@ 0000000180005008     libisfldsin003.obj
 0002:00001020       ??_C@_0BF@OLIHJOII@JVMTI_ERROR_INTERNAL@ 0000000180005020     libisfldsin003.obj
 0002:00001038       ??_C@_0BO@EOHGKJHI@JVMTI_ERROR_UNATTACHED_THREAD@ 0000000180005038     libisfldsin003.obj
 0002:00001058       ??_C@_0CA@LKHFDACL@JVMTI_ERROR_INVALID_ENVIRONMENT@ 0000000180005058     libisfldsin003.obj
 0002:00001078       ??_C@_0BA@MMFHLOKK@?$DMunknown?5error?$DO@ 0000000180005078     libisfldsin003.obj
 0002:00001088       ??_C@_0CF@CBHOKDB@throwable?5?$DN?5jni?9?$DOExceptionOccur@ 0000000180005088     libisfldsin003.obj
 0002:000010b0       ??_C@_03OFAPEBGM@?$CFs?6@  00000001800050b0     libisfldsin003.obj
 0002:000010b8       ??_C@_0DM@LPIGEGNJ@s?2test?2hotspot?2jtreg?2vmTestbase@ 00000001800050b8     libisfldsin003.obj
 0002:000010f8       ??_C@_0CC@NFCNPEPK@Exception?5in?5JNI?5call?5?$CIcleared?$CJ@ 00000001800050f8     libisfldsin003.obj
 0002:00001120       ??_C@_0BJ@IBAKFIKF@jni?9?$DOExceptionDescribe?$CI?$CJ@ 0000000180005120     libisfldsin003.obj
 0002:00001140       ??_C@_0BG@GGKALKMH@jni?9?$DOExceptionClear?$CI?$CJ@ 0000000180005140     libisfldsin003.obj
 0002:00001158       ??_C@_0CF@JMGFGJLJ@?$CD?5?5?5verified?5JNI?5assertion?5is?5F@ 0000000180005158     libisfldsin003.obj
 0002:00001180       ??_C@_0CB@MLNJNCLJ@?5?5jvmti?5error?3?5code?$DN?$CFd?0?5name?$DN?$CFs@ 0000000180005180     libisfldsin003.obj
 0002:000011a8       ??_C@_0CD@OHBGDKMK@?$CD?5?5?5jvmti?5error?3?5code?$DN?$CFd?0?5name?$DN@ 00000001800051a8     libisfldsin003.obj
 0002:000011d0       ??_C@_0CG@JNNCGPHB@?$CD?5?5?5error?5expected?3?5code?$DN?$CFd?0?5na@ 00000001800051d0     libisfldsin003.obj
 0002:00001200       ??_C@_0EB@IMGKPCGE@?$CIstr_obj?5?$DN?5jni?9?$DONewStringUTF?$CIco@ 0000000180005200     libisfldsin003.obj
 0002:00001250       ??_C@_0EA@HFOGGBCC@s?2test?2hotspot?2jtreg?2vmTestbase@ 0000000180005250     libisfldsin003.obj
 0002:00001290       ??_C@_05KKCIMGE@error@     0000000180005290     libisfldsin003.obj
 0002:00001298       ??_C@_0CJ@JACLEAA@Test?5failed?5by?5setFailStatus?$CI?$CJ?4@ 0000000180005298     libisfldsin003.obj
 0002:000012d0       ??_C@_0EA@PNBCDMOA@s?2test?2hotspot?2jtreg?2vmTestbase@ 00000001800052d0     libisfldsin003.obj
 0002:00001310       ??_C@_0DI@ILAHDLMP@?$CI?$CKagentThreadProc?$CJ?$CIjvmti_env?0?5a@ 0000000180005310     libisfldsin003.obj
 0002:00001348       ??_C@_0BD@KDBALNLB@JVMTI?5agent?5thread@ 0000000180005348     libisfldsin003.obj
 0002:00001360       ??_C@_0BB@NOKBFPFO@java?1lang?1Thread@ 0000000180005360     libisfldsin003.obj
 0002:00001374       ??_C@_06FALKBLGB@?$DMinit?$DO@ 0000000180005374     libisfldsin003.obj
 0002:00001380       ??_C@_0BG@IKDDPPGD@?$CILjava?1lang?1String?$DL?$CJV@ 0000000180005380     libisfldsin003.obj
 0002:000013a0       ??_C@_0EB@IFJBFEKC@?$CIthreadClass?5?$DN?5jni_env?9?$DOFindCla@ 00000001800053a0     libisfldsin003.obj
 0002:000013f0       ??_C@_0GF@FGFIBKKL@?$CIthreadCtor?5?$DN?5jni_env?9?$DOGetMetho@ 00000001800053f0     libisfldsin003.obj
 0002:00001458       ??_C@_0DN@NCPDJLOG@?$CIthreadName?5?$DN?5jni_env?9?$DONewStrin@ 0000000180005458     libisfldsin003.obj
 0002:000014a0       ??_C@_0FE@PFKODBGC@?$CIthreadObject?5?$DN?5jni_env?9?$DONewObj@ 00000001800054a0     libisfldsin003.obj
 0002:00001500       ??_C@_0ED@HOBAHHJI@?$CIthreadGlobalRef?5?$DN?5jni_env?9?$DONew@ 0000000180005500     libisfldsin003.obj
 0002:00001550       ??_C@_0FN@HNJJAHFC@jvmti_env?9?$DORunAgentThread?$CIagent@ 0000000180005550     libisfldsin003.obj
 0002:000015b0       ??_C@_0EA@MOJDNKDF@Debuggee?5status?5sync?5aborted?5be@ 00000001800055b0     libisfldsin003.obj
 0002:000015f0       ??_C@_0EA@EEOEJAEN@status?5?$DN?5syncDebuggeeStatus?$CIjni@ 00000001800055f0     libisfldsin003.obj
 0002:00001630       ??_C@_0BL@JBCFNBMB@nsk_jvmti_resetAgentData?$CI?$CJ@ 0000000180005630     libisfldsin003.obj
 0002:00001650       ??_C@_0EL@LPBEELIP@s?2test?2hotspot?2jtreg?2vmTestbase@ 0000000180005650     libisfldsin003.obj
 0002:000016a0       ??_C@_0CK@JDAMFDMJ@jvmti?9?$DOSetTag?$CIo?0?5tag?$CJ?5?$DN?$DN?5JVMTI_@ 00000001800056a0     libisfldsin003.obj
 0002:000016d0       ??_C@_0CC@DAMNHKNI@Can?8t?5set?5tag?5?$CFli?5for?5object?5?$CFl@ 00000001800056d0     libisfldsin003.obj
 0002:000016f8       ??_C@_0DL@HAJPNKEF@jvmti?9?$DOGetObjectHashCode?$CIo?0?5?$CGha@ 00000001800056f8     libisfldsin003.obj
 0002:00001738       ??_C@_0BL@JFPIEOBF@Can?8t?5get?5hash?5object?5?$CFlx?6@ 0000000180005738     libisfldsin003.obj
 0002:00001758       ??_C@_0BG@DICPHBKN@setTag?3?5?$CF08x?5?$DM?9?5?$CF?53li@ 0000000180005758     libisfldsin003.obj
 0002:00001770       ??_C@_0DH@FCEEBDMJ@?$CIs?5?$DN?5jni?9?$DOGetStringUTFChars?$CIsIn@ 0000000180005770     libisfldsin003.obj
 0002:000017a8       ??_C@_0BJ@OKKGHDCN@Can?8t?5get?5string?5at?5?$CF?$CDp?6@ 00000001800057a8     libisfldsin003.obj
 0002:000017c8       ??_C@_0BP@EKFLGGFJ@Can?8t?5get?5string?5at?5?$CF?$CDp?3?5null?6@ 00000001800057c8     libisfldsin003.obj
 0002:000017e8       ??_C@_06ICODBHCL@?5?1?1?5?$CFs@ 00000001800057e8     libisfldsin003.obj
 0002:000017f0       ??_C@_0DB@KGFPLEGO@?$CIr?5?$DN?5jvmti?9?$DOGetTag?$CIo?0?5?$CGtag?$CJ?$CJ?5?$DN?$DN@ 00000001800057f0     libisfldsin003.obj
 0002:00001828       ??_C@_0CO@PDAGBCGJ@Can?8t?5GetTag?5for?5object?5?$CFlx?4?5Re@ 0000000180005828     libisfldsin003.obj
 0002:00001858       ??_C@_0CH@HPEODOHC@TEST_BUG?3?5Max?4?5number?5of?5refs?5r@ 0000000180005858     libisfldsin003.obj
 0002:00001880       ??_C@_0DI@PHFCABIM@?$CIr?5?$DN?5jvmti?9?$DOGetTag?$CIfrom?0?5?$CGtagFr@ 0000000180005880     libisfldsin003.obj
 0002:000018b8       ??_C@_0DI@MDEGFNKD@TEST_BUG?3?5Can?8t?5GetTag?5for?5obje@ 00000001800058b8     libisfldsin003.obj
 0002:000018f0       ??_C@_0DE@MLELJAHM@?$CIr?5?$DN?5jvmti?9?$DOGetTag?$CIto?0?5?$CGtagTo?$CJ?$CJ@ 00000001800058f0     libisfldsin003.obj
 0002:00001928       ??_C@_09OPJEJKBL@printdump@ 0000000180005928     libisfldsin003.obj
 0002:00001938       ??_C@_0CJ@KCDEKOCJ@Wrong?5result?5of?5a?5valid?5call?5to@ 0000000180005938     libisfldsin003.obj
 0002:00001968       ??_C@_0DG@LAJPGIIE@?$CIGetPotentialCapabilities?$CJ?5unex@ 0000000180005968     libisfldsin003.obj
 0002:000019a0       ??_C@_0CN@LKPEOJPO@?$CIAddCapabilities?$CJ?5unexpected?5er@ 00000001800059a0     libisfldsin003.obj
 0002:000019d0       ??_C@_0CN@BCCBOHCH@?$CIGetCapabilities?$CJ?5unexpected?5er@ 00000001800059d0     libisfldsin003.obj
 0002:00001a00       ??_C@_0CO@GFLJNBP@Warning?3?5IsFieldSynthetic?5is?5no@ 0000000180005a00     libisfldsin003.obj
 0002:00001a30       ??_C@_04LOAJBDKD@true@     0000000180005a30     libisfldsin003.obj
 0002:00001a38       ??_C@_05LAPONLG@false@     0000000180005a38     libisfldsin003.obj
 0002:00001a40       ??_C@_0CH@CDOJMNAO@JVMTI?5client?5was?5not?5properly?5l@ 0000000180005a40     libisfldsin003.obj
 0002:00001a68       ??_C@_0CI@HIFAHBMG@?$CI?$CFllu?$CJ?5cannot?5get?5field?5ID?5for?5@ 0000000180005a68     libisfldsin003.obj
 0002:00001a90       ??_C@_0DD@HJCHHDD@?$CIIsFieldSynthetic?$CD?$CFllu?$CJ?5unexpec@ 0000000180005a90     libisfldsin003.obj
 0002:00001ac8       ??_C@_0BO@FFEEPNJ@?$DO?$DO?$DO?5?$CFs?3?$CC?$CFs?$CC?0?5isSynthetic?3?5?$CFs?6@ 0000000180005ac8     libisfldsin003.obj
 0002:00001ae8       ??_C@_0DC@MAPINGDG@?$CFs?3?$CC?$CFs?$CC?6?7?5?9?5isSynthetic?5expecte@ 0000000180005ae8     libisfldsin003.obj
 0002:00001b30       ??_C@_1EC@JIJBPKFM@?$AAa?$AAp?$AAi?$AA?9?$AAm?$AAs?$AA?9?$AAw?$AAi?$AAn?$AA?9?$AAc?$AAo?$AAr?$AAe@ 0000000180005b30     MSVCRT:thread_safe_statics.obj
 0002:00001b78       ??_C@_1BK@MGMFAEKH@?$AAk?$AAe?$AAr?$AAn?$AAe?$AAl?$AA3?$AA2?$AA?4?$AAd?$AAl?$AAl@ 0000000180005b78     MSVCRT:thread_safe_statics.obj
 0002:00001b98       ??_C@_0BJ@JEBJOJFJ@SleepConditionVariableCS@ 0000000180005b98     MSVCRT:thread_safe_statics.obj
 0002:00001bb8       ??_C@_0BJ@PGPPEPCC@WakeAllConditionVariable@ 0000000180005bb8     MSVCRT:thread_safe_statics.obj
 0002:00001bd8       _pDefaultRawDllMain        0000000180005bd8     MSVCRT:dll_dllmain.obj
 0002:00001bd8       _pRawDllMain               0000000180005bd8     MSVCRT:dll_dllmain.obj
 0002:00001be0       __xmm@ffffffffffffffffffffffffffffffff 0000000180005be0     MSVCRT:utility.obj
 0002:00001bf0       _load_config_used          0000000180005bf0     MSVCRT:loadcfg.obj
 0002:00001e00       _tls_used                  0000000180005e00     MSVCRT:tlssup.obj
 0002:00001e28       __volatile_metadata        0000000180005e28     <linker-defined>
 0002:000021e8       __rtc_iaa                  00000001800061e8     MSVCRT:initsect.obj
 0002:000021f0       __rtc_izz                  00000001800061f0     MSVCRT:initsect.obj
 0002:000021f8       __rtc_taa                  00000001800061f8     MSVCRT:initsect.obj
 0002:00002200       __rtc_tzz                  0000000180006200     MSVCRT:initsect.obj
 0002:00002208       _tls_start                 0000000180006208     MSVCRT:tlssup.obj
 0002:0000220c       _Init_thread_epoch         000000018000620c     MSVCRT:thread_safe_statics.obj
 0002:00002210       _tls_end                   0000000180006210     MSVCRT:tlssup.obj
 0002:000028a0       __IMPORT_DESCRIPTOR_KERNEL32 00000001800068a0     kernel32:KERNEL32.dll
 0002:000028b4       __IMPORT_DESCRIPTOR_VCRUNTIME140 00000001800068b4     vcruntime:VCRUNTIME140.dll
 0002:000028c8       __IMPORT_DESCRIPTOR_api-ms-win-crt-runtime-l1-1-0 00000001800068c8     ucrt:api-ms-win-crt-runtime-l1-1-0.dll
 0002:000028dc       __IMPORT_DESCRIPTOR_api-ms-win-crt-stdio-l1-1-0 00000001800068dc     ucrt:api-ms-win-crt-stdio-l1-1-0.dll
 0002:000028f0       __IMPORT_DESCRIPTOR_api-ms-win-crt-string-l1-1-0 00000001800068f0     ucrt:api-ms-win-crt-string-l1-1-0.dll
 0002:00002904       __NULL_IMPORT_DESCRIPTOR   0000000180006904     kernel32:KERNEL32.dll
 0003:00000060       _Init_global_epoch         0000000180007060     MSVCRT:thread_safe_statics.obj
 0003:00000070       __security_cookie          0000000180007070     MSVCRT:gs_cookie.obj
 0003:00000078       __security_cookie_complement 0000000180007078     MSVCRT:gs_cookie.obj
 0003:00000080       __scrt_native_dllmain_reason 0000000180007080     MSVCRT:utility.obj
 0003:00000088       __isa_available            0000000180007088     MSVCRT:cpu_disp.obj
 0003:0000008c       __isa_enabled              000000018000708c     MSVCRT:cpu_disp.obj
 0003:00000090       __memset_fast_string_threshold 0000000180007090     MSVCRT:cpu_disp.obj
 0003:00000098       __memset_nt_threshold      0000000180007098     MSVCRT:cpu_disp.obj
 0003:000000a0       __scrt_ucrt_dll_is_in_use  00000001800070a0     MSVCRT:ucrt_stubs.obj
 0003:000000b0       g_wrongHeapCallbacks       00000001800070b0     libisfldsin003.obj
 0003:00000130       g_szTagInfo                0000000180007130     libisfldsin003.obj
 0003:00002070       g_tagFlags                 0000000180009070     libisfldsin003.obj
 0003:00002458       g_refsToVerifyCnt          0000000180009458     libisfldsin003.obj
 0003:0000245c       g_fakeUserData             000000018000945c     libisfldsin003.obj
 0003:00002460       g_tagVisitCount            0000000180009460     libisfldsin003.obj
 0003:00003400       g_refsToVerify             000000018000a400     libisfldsin003.obj
 0003:0001ab00       g_userDataError            0000000180021b00     libisfldsin003.obj
 0003:0001acb0       ?_OptionsStorage@?1??__local_stdio_printf_options@@9@4_KA 0000000180021cb0     libisfldsin003.obj
 0003:0001b278       _tls_index                 0000000180022278     MSVCRT:tlssup.obj
 0003:0001b280       __scrt_current_native_startup_state 0000000180022280     MSVCRT:utility.obj
 0003:0001b288       __scrt_native_startup_lock 0000000180022288     MSVCRT:utility.obj
 0003:0001b2c8       __scrt_debugger_hook_flag  00000001800222c8     MSVCRT:utility_desktop.obj
 0003:0001b2d0       ?__type_info_root_node@@3U__type_info_node@@A 00000001800222d0     MSVCRT:tncleanup.obj
 0003:0001b2e0       ?_OptionsStorage@?1??__local_stdio_scanf_options@@9@4_KA 00000001800222e0     MSVCRT:default_local_stdio_options.obj
 0003:0001b2e8       __favor                    00000001800222e8     MSVCRT:cpu_disp.obj
 0003:0001b2f0       __dyn_tls_init_callback    00000001800222f0     <common>

 entry point at        0001:00002310

 Static symbols

 0000:fffdb000       .debug$S                   0000000180000000     isfldsin003.exp
 0000:fffdb000       .debug$S                   0000000180000000     vcruntime:VCRUNTIME140.dll
 0000:fffdb000       .debug$S                   0000000180000000     vcruntime:VCRUNTIME140.dll
 0000:fffdb000       .debug$S                   0000000180000000     vcruntime:VCRUNTIME140.dll
 0000:fffdb000       .debug$S                   0000000180000000     vcruntime:VCRUNTIME140.dll
 0000:fffdb000       .debug$S                   0000000180000000     vcruntime:VCRUNTIME140.dll
 0000:fffdb000       .debug$S                   0000000180000000     vcruntime:VCRUNTIME140.dll
 0000:fffdb000       .debug$S                   0000000180000000     vcruntime:VCRUNTIME140.dll
 0000:fffdb000       .debug$S                   0000000180000000     ucrt:api-ms-win-crt-convert-l1-1-0.dll
 0002:ffffc000       .idata$6                   0000000180000000     ucrt:api-ms-win-crt-convert-l1-1-0.dll
 0000:fffdb000       .debug$S                   0000000180000000     ucrt:api-ms-win-crt-heap-l1-1-0.dll
 0000:fffdb000       .debug$S                   0000000180000000     ucrt:api-ms-win-crt-heap-l1-1-0.dll
 0000:fffdb000       .debug$S                   0000000180000000     ucrt:api-ms-win-crt-heap-l1-1-0.dll
 0000:fffdb000       .debug$S                   0000000180000000     ucrt:api-ms-win-crt-heap-l1-1-0.dll
 0002:ffffc000       .idata$6                   0000000180000000     ucrt:api-ms-win-crt-heap-l1-1-0.dll
 0000:fffdb000       .debug$S                   0000000180000000     ucrt:api-ms-win-crt-runtime-l1-1-0.dll
 0000:fffdb000       .debug$S                   0000000180000000     ucrt:api-ms-win-crt-runtime-l1-1-0.dll
 0000:fffdb000       .debug$S                   0000000180000000     ucrt:api-ms-win-crt-runtime-l1-1-0.dll
 0000:fffdb000       .debug$S                   0000000180000000     ucrt:api-ms-win-crt-runtime-l1-1-0.dll
 0000:fffdb000       .debug$S                   0000000180000000     ucrt:api-ms-win-crt-runtime-l1-1-0.dll
 0000:fffdb000       .debug$S                   0000000180000000     ucrt:api-ms-win-crt-runtime-l1-1-0.dll
 0000:fffdb000       .debug$S                   0000000180000000     ucrt:api-ms-win-crt-runtime-l1-1-0.dll
 0000:fffdb000       .debug$S                   0000000180000000     ucrt:api-ms-win-crt-runtime-l1-1-0.dll
 0000:fffdb000       .debug$S                   0000000180000000     ucrt:api-ms-win-crt-runtime-l1-1-0.dll
 0000:fffdb000       .debug$S                   0000000180000000     ucrt:api-ms-win-crt-runtime-l1-1-0.dll
 0000:fffdb000       .debug$S                   0000000180000000     ucrt:api-ms-win-crt-runtime-l1-1-0.dll
 0000:fffdb000       .debug$S                   0000000180000000     ucrt:api-ms-win-crt-runtime-l1-1-0.dll
 0000:fffdb000       .debug$S                   0000000180000000     ucrt:api-ms-win-crt-runtime-l1-1-0.dll
 0000:fffdb000       .debug$S                   0000000180000000     ucrt:api-ms-win-crt-runtime-l1-1-0.dll
 0000:fffdb000       .debug$S                   0000000180000000     ucrt:api-ms-win-crt-runtime-l1-1-0.dll
 0000:fffdb000       .debug$S                   0000000180000000     ucrt:api-ms-win-crt-runtime-l1-1-0.dll
 0000:fffdb000       .debug$S                   0000000180000000     ucrt:api-ms-win-crt-stdio-l1-1-0.dll
 0000:fffdb000       .debug$S                   0000000180000000     ucrt:api-ms-win-crt-stdio-l1-1-0.dll
 0000:fffdb000       .debug$S                   0000000180000000     ucrt:api-ms-win-crt-stdio-l1-1-0.dll
 0000:fffdb000       .debug$S                   0000000180000000     ucrt:api-ms-win-crt-stdio-l1-1-0.dll
 0000:fffdb000       .debug$S                   0000000180000000     ucrt:api-ms-win-crt-stdio-l1-1-0.dll
 0000:fffdb000       .debug$S                   0000000180000000     ucrt:api-ms-win-crt-stdio-l1-1-0.dll
 0000:fffdb000       .debug$S                   0000000180000000     ucrt:api-ms-win-crt-stdio-l1-1-0.dll
 0000:fffdb000       .debug$S                   0000000180000000     ucrt:api-ms-win-crt-stdio-l1-1-0.dll
 0000:fffdb000       .debug$S                   0000000180000000     ucrt:api-ms-win-crt-stdio-l1-1-0.dll
 0000:fffdb000       .debug$S                   0000000180000000     ucrt:api-ms-win-crt-stdio-l1-1-0.dll
 0000:fffdb000       .debug$S                   0000000180000000     ucrt:api-ms-win-crt-string-l1-1-0.dll
 0000:fffdb000       .debug$S                   0000000180000000     ucrt:api-ms-win-crt-string-l1-1-0.dll
 0000:fffdb000       .debug$S                   0000000180000000     ucrt:api-ms-win-crt-string-l1-1-0.dll
 0000:fffdb000       .debug$S                   0000000180000000     ucrt:api-ms-win-crt-string-l1-1-0.dll
 0000:fffdb000       .debug$S                   0000000180000000     ucrt:api-ms-win-crt-string-l1-1-0.dll
 0000:fffdb000       .debug$S                   0000000180000000     ucrt:api-ms-win-crt-string-l1-1-0.dll
 0000:fffdb000       .debug$S                   0000000180000000     ucrt:api-ms-win-crt-string-l1-1-0.dll
 0000:fffdb000       .debug$S                   0000000180000000     ucrt:api-ms-win-crt-string-l1-1-0.dll
 0000:fffdb000       .debug$S                   0000000180000000     kernel32:KERNEL32.dll
 0000:fffdb000       .debug$S                   0000000180000000     kernel32:KERNEL32.dll
 0000:fffdb000       .debug$S                   0000000180000000     kernel32:KERNEL32.dll
 0000:fffdb000       .debug$S                   0000000180000000     kernel32:KERNEL32.dll
 0000:fffdb000       .debug$S                   0000000180000000     kernel32:KERNEL32.dll
 0000:fffdb000       .debug$S                   0000000180000000     kernel32:KERNEL32.dll
 0000:fffdb000       .debug$S                   0000000180000000     kernel32:KERNEL32.dll
 0000:fffdb000       .debug$S                   0000000180000000     kernel32:KERNEL32.dll
 0000:fffdb000       .debug$S                   0000000180000000     kernel32:KERNEL32.dll
 0000:fffdb000       .debug$S                   0000000180000000     kernel32:KERNEL32.dll
 0000:fffdb000       .debug$S                   0000000180000000     kernel32:KERNEL32.dll
 0000:fffdb000       .debug$S                   0000000180000000     kernel32:KERNEL32.dll
 0000:fffdb000       .debug$S                   0000000180000000     kernel32:KERNEL32.dll
 0000:fffdb000       .debug$S                   0000000180000000     kernel32:KERNEL32.dll
 0000:fffdb000       .debug$S                   0000000180000000     kernel32:KERNEL32.dll
 0000:fffdb000       .debug$S                   0000000180000000     kernel32:KERNEL32.dll
 0000:fffdb000       .debug$S                   0000000180000000     kernel32:KERNEL32.dll
 0000:fffdb000       .debug$S                   0000000180000000     kernel32:KERNEL32.dll
 0000:fffdb000       .debug$S                   0000000180000000     kernel32:KERNEL32.dll
 0000:fffdb000       .debug$S                   0000000180000000     kernel32:KERNEL32.dll
 0000:fffdb000       .debug$S                   0000000180000000     kernel32:KERNEL32.dll
 0000:fffdb000       .debug$S                   0000000180000000     kernel32:KERNEL32.dll
 0000:fffdb000       .debug$S                   0000000180000000     kernel32:KERNEL32.dll
 0000:fffdb000       .debug$S                   0000000180000000     kernel32:KERNEL32.dll
 0000:fffdb000       .debug$S                   0000000180000000     kernel32:KERNEL32.dll
 0000:fffdb000       .debug$S                   0000000180000000     kernel32:KERNEL32.dll
 0000:fffdb000       .debug$S                   0000000180000000     kernel32:KERNEL32.dll
 0000:fffdb000       .debug$S                   0000000180000000     kernel32:KERNEL32.dll
 0001:00000f2c       addRefToVerify             0000000180001f2c f   libisfldsin003.obj
 0001:00000f98       agentThreadWrapper         0000000180001f98 f   libisfldsin003.obj
 0001:00001188       file_basename              0000000180002188 f   libisfldsin003.obj
 0001:000017f4       startAgentThreadWrapper    00000001800027f4 f   libisfldsin003.obj
 0001:00001b34       syncDebuggeeStatus         0000000180002b34 f   libisfldsin003.obj
 0001:00001dd4       capture_previous_context   0000000180002dd4 f   MSVCRT:gs_report.obj
 0001:00001e48       ?__scrt_initialize_thread_safe_statics@@YAHXZ 0000000180002e48 f   MSVCRT:thread_safe_statics.obj
 0001:00001f18       ?__scrt_uninitialize_thread_safe_statics@@YAXXZ 0000000180002f18 f   MSVCRT:thread_safe_statics.obj
 0001:00001fc0       $$000000                   0000000180002fc0     MSVCRT:amdsecgs.obj
 0001:00001ff0       ?dllmain_crt_dispatch@@YAHQEAUHINSTANCE__@@KQEAX@Z 0000000180002ff0 f   MSVCRT:dll_dllmain.obj
 0001:00002040       ?dllmain_crt_process_attach@@YAHQEAUHINSTANCE__@@QEAX@Z 0000000180003040 f   MSVCRT:dll_dllmain.obj
 0001:00002158       ?dllmain_crt_process_detach@@YAH_N@Z 0000000180003158 f   MSVCRT:dll_dllmain.obj
 0001:000021dc       ?dllmain_dispatch@@YAHQEAUHINSTANCE__@@KQEAX@Z 00000001800031dc f   MSVCRT:dll_dllmain.obj
 0001:00002bf0       $$000000                   0000000180003bf0     MSVCRT:guard_dispatch.obj
 0001:00002c10       $$000000                   0000000180003c10     MSVCRT:guard_xfg_dispatch.obj
 0001:00002c26       ?fin$0@?0??dllmain_crt_process_attach@@YAHQEAUHINSTANCE__@@QEAX@Z@4HA 0000000180003c26 f   MSVCRT:dll_dllmain.obj
 0001:00002c3d       ?fin$0@?0??dllmain_crt_process_detach@@YAH_N@Z@4HA 0000000180003c3d f   MSVCRT:dll_dllmain.obj
 0001:00002c56       ?fin$1@?0??dllmain_crt_process_detach@@YAH_N@Z@4HA 0000000180003c56 f   MSVCRT:dll_dllmain.obj
 0001:00002c6a       ?filt$0@?0??dllmain_dispatch@@YAHQEAUHINSTANCE__@@KQEAX@Z@4HA 0000000180003c6a f   MSVCRT:dll_dllmain.obj
 0001:00002ca0       __scrt_is_nonwritable_in_current_image$filt$0 0000000180003ca0 f   MSVCRT:utility.obj
 0002:000001e8       ?__scrt_initialize_tss_var@@3P6AHXZEA 00000001800041e8     MSVCRT:thread_safe_statics.obj
 0002:00000310       ?opcLengths@@3QBEB         0000000180004310     libisfldsin003.obj
 0002:00001b20       GS_ExceptionPointers       0000000180005b20     MSVCRT:gs_report.obj
 0002:00002218       $unwind$fprintf            0000000180006218     libisfldsin003.obj
 0002:00002224       $unwind$printf             0000000180006224     libisfldsin003.obj
 0002:00002230       $unwind$?NewObject@JNIEnv_@@QEAAPEAV_jobject@@PEAV_jclass@@PEAU_jmethodID@@ZZ 0000000180006230     libisfldsin003.obj
 0002:00002230       $unwind$nsk_lcomplain      0000000180006230     libisfldsin003.obj
 0002:00002230       $unwind$nsk_ldisplay       0000000180006230     libisfldsin003.obj
 0002:00002238       $unwind$nsk_lvdisplay      0000000180006238     libisfldsin003.obj
 0002:00002238       $unwind$_RTC_Initialize    0000000180006238     MSVCRT:initsect.obj
 0002:00002238       $unwind$_RTC_Terminate     0000000180006238     MSVCRT:initsect.obj
 0002:00002238       $unwind$?__scrt_initialize_thread_safe_statics@@YAHXZ 0000000180006238     MSVCRT:thread_safe_statics.obj
 0002:00002244       $unwind$nsk_lvcomplain     0000000180006244     libisfldsin003.obj
 0002:0000225c       $unwind$nsk_ltrace         000000018000625c     libisfldsin003.obj
 0002:0000225c       $unwind$__report_gsfailure 000000018000625c     MSVCRT:gs_report.obj
 0002:00002264       $unwind$Agent_Initialize   0000000180006264     libisfldsin003.obj
 0002:00002264       $unwind$nsk_lvtrace        0000000180006264     libisfldsin003.obj
 0002:00002264       $unwind$__raise_securityfailure 0000000180006264     MSVCRT:gs_report.obj
 0002:00002264       $unwind$__scrt_initialize_crt 0000000180006264     MSVCRT:utility.obj
 0002:00002264       $unwind$__scrt_initialize_onexit_tables 0000000180006264     MSVCRT:utility.obj
 0002:00002264       $unwind$__scrt_release_startup_lock 0000000180006264     MSVCRT:utility.obj
 0002:00002264       $unwind$__scrt_uninitialize_crt 0000000180006264     MSVCRT:utility.obj
 0002:00002264       $unwind$_onexit            0000000180006264     MSVCRT:utility.obj
 0002:0000226c       $unwind$nsk_lverify        000000018000626c     libisfldsin003.obj
 0002:0000227c       $unwind$nsk_vprintf        000000018000627c     libisfldsin003.obj
 0002:0000228c       $unwind$nsk_printf         000000018000628c     libisfldsin003.obj
 0002:00002294       $unwind$?nsk_jni_lverify@@YAHHPEAUJNIEnv_@@HQEBDH1ZZ 0000000180006294     libisfldsin003.obj
 0002:000022a8       $unwind$?nsk_jni_check_exception@@YAHPEAUJNIEnv_@@QEBDH@Z 00000001800062a8     libisfldsin003.obj
 0002:000022c4       $unwind$Java_nsk_jvmti_unit_FollowReferences_FollowRefObjects_resetTags 00000001800062c4     libisfldsin003.obj
 0002:000022c4       $unwind$addRefToVerify     00000001800062c4     libisfldsin003.obj
 0002:000022c4       $unwind$nsk_jvmti_resetAgentData 00000001800062c4     libisfldsin003.obj
 0002:000022c4       $unwind$nsk_jvmti_setFailStatus 00000001800062c4     libisfldsin003.obj
 0002:000022c4       $unwind$__scrt_initialize_default_local_stdio_options 00000001800062c4     MSVCRT:default_local_stdio_options.obj
 0002:000022c4       $unwind$?dllmain_crt_dispatch@@YAHQEAUHINSTANCE__@@KQEAX@Z 00000001800062c4     MSVCRT:dll_dllmain.obj
 0002:000022c4       $unwind$DllMain            00000001800062c4     MSVCRT:dll_dllmain_stub.obj
 0002:000022c4       $unwind$__GSHandlerCheck   00000001800062c4     MSVCRT:gshandler.obj
 0002:000022c4       $unwind$?__scrt_uninitialize_thread_safe_statics@@YAXXZ 00000001800062c4     MSVCRT:thread_safe_statics.obj
 0002:000022c4       $unwind$__scrt_acquire_startup_lock 00000001800062c4     MSVCRT:utility.obj
 0002:000022c4       $unwind$__scrt_dllmain_after_initialize_c 00000001800062c4     MSVCRT:utility.obj
 0002:000022c4       $unwind$__scrt_dllmain_before_initialize_c 00000001800062c4     MSVCRT:utility.obj
 0002:000022c4       $unwind$__scrt_dllmain_crt_thread_attach 00000001800062c4     MSVCRT:utility.obj
 0002:000022c4       $unwind$__scrt_dllmain_crt_thread_detach 00000001800062c4     MSVCRT:utility.obj
 0002:000022c4       $unwind$__scrt_dllmain_uninitialize_c 00000001800062c4     MSVCRT:utility.obj
 0002:000022c4       $unwind$__scrt_dllmain_uninitialize_critical 00000001800062c4     MSVCRT:utility.obj
 0002:000022c4       $unwind$atexit             00000001800062c4     MSVCRT:utility.obj
 0002:000022cc       $unwind$nsk_jvmti_lverify  00000001800062cc     libisfldsin003.obj
 0002:000022e0       $unwind$exitOnError        00000001800062e0     libisfldsin003.obj
 0002:000022f0       $unwind$Java_nsk_share_jvmti_ArgumentHandler_getAgentOptionsString 00000001800062f0     libisfldsin003.obj
 0002:00002304       $unwind$Java_nsk_jvmti_unit_FollowReferences_FollowRefObjects_getTag 0000000180006304     libisfldsin003.obj
 0002:00002304       $unwind$Java_nsk_share_jvmti_DebugeeClass_checkStatus 0000000180006304     libisfldsin003.obj
 0002:00002304       $unwind$agentThreadWrapper 0000000180006304     libisfldsin003.obj
 0002:00002314       $unwind$startAgentThreadWrapper 0000000180006314     libisfldsin003.obj
 0002:00002330       $unwind$syncDebuggeeStatus 0000000180006330     libisfldsin003.obj
 0002:00002330       $unwind$__scrt_dllmain_exception_filter 0000000180006330     MSVCRT:utility.obj
 0002:00002344       $unwind$Java_nsk_share_jvmti_DebugeeClass_resetAgentData 0000000180006344     libisfldsin003.obj
 0002:0000234c       $unwind$MA_checkStatus     000000018000634c     libisfldsin003.obj
 0002:00002360       $unwind$Java_nsk_jvmti_unit_FollowReferences_FollowRefObjects_setTag 0000000180006360     libisfldsin003.obj
 0002:00002378       $unwind$Java_nsk_jvmti_unit_FollowReferences_FollowRefObjects_addRefToVerify 0000000180006378     libisfldsin003.obj
 0002:00002394       $unwind$Java_nsk_jvmti_IsFieldSynthetic_isfldsin003a_check 0000000180006394     libisfldsin003.obj
 0002:000023ac       $unwind$capture_previous_context 00000001800063ac     MSVCRT:gs_report.obj
 0002:000023b8       $unwind$__GSHandlerCheckCommon 00000001800063b8     MSVCRT:gshandler.obj
 0002:000023c0       $xdatasym                  00000001800063c0     MSVCRT:amdsecgs.obj
 0002:000023c4       $unwind$?dllmain_crt_process_attach@@YAHQEAUHINSTANCE__@@QEAX@Z 00000001800063c4     MSVCRT:dll_dllmain.obj
 0002:00002400       $unwind$?fin$0@?0??dllmain_crt_process_attach@@YAHQEAUHINSTANCE__@@QEAX@Z@4HA 0000000180006400     MSVCRT:dll_dllmain.obj
 0002:00002400       $unwind$?fin$0@?0??dllmain_crt_process_detach@@YAH_N@Z@4HA 0000000180006400     MSVCRT:dll_dllmain.obj
 0002:00002400       $unwind$?fin$1@?0??dllmain_crt_process_detach@@YAH_N@Z@4HA 0000000180006400     MSVCRT:dll_dllmain.obj
 0002:00002408       $unwind$?dllmain_crt_process_detach@@YAH_N@Z 0000000180006408     MSVCRT:dll_dllmain.obj
 0002:0000245c       $unwind$?dllmain_dispatch@@YAHQEAUHINSTANCE__@@KQEAX@Z 000000018000645c     MSVCRT:dll_dllmain.obj
 0002:00002484       $unwind$?filt$0@?0??dllmain_dispatch@@YAHQEAUHINSTANCE__@@KQEAX@Z@4HA 0000000180006484     MSVCRT:dll_dllmain.obj
 0002:0000248c       $unwind$_DllMainCRTStartup 000000018000648c     MSVCRT:dll_dllmain.obj
 0002:0000249c       $unwind$__scrt_is_nonwritable_in_current_image 000000018000649c     MSVCRT:utility.obj
 0002:000024bc       $unwind$__scrt_is_nonwritable_in_current_image$filt$0 00000001800064bc     MSVCRT:utility.obj
 0002:000024c4       $unwind$__scrt_fastfail    00000001800064c4     MSVCRT:utility_desktop.obj
 0002:000024d4       $unwind$__security_init_cookie 00000001800064d4     MSVCRT:gs_support.obj
 0002:000024e0       $unwind$__isa_available_init 00000001800064e0     MSVCRT:cpu_disp.obj
 0002:000024f0       $xdatasym                  00000001800064f0     MSVCRT:guard_dispatch.obj
 0002:000024f8       $xdatasym                  00000001800064f8     MSVCRT:guard_xfg_dispatch.obj
 0002:00002500       .edata                     0000000180006500     isfldsin003.exp
 0002:00002528       rgpv                       0000000180006528     isfldsin003.exp
 0002:00002564       rgszName                   0000000180006564     isfldsin003.exp
 0002:000025a0       rgwOrd                     00000001800065a0     isfldsin003.exp
 0002:000025be       szName                     00000001800065be     isfldsin003.exp
 0002:000025ce       $N00001                    00000001800065ce     isfldsin003.exp
 0002:000025dd       $N00002                    00000001800065dd     isfldsin003.exp
 0002:000025ea       $N00003                    00000001800065ea     isfldsin003.exp
 0002:0000261d       $N00004                    000000018000661d     isfldsin003.exp
 0002:00002662       $N00005                    0000000180006662     isfldsin003.exp
 0002:0000269f       $N00006                    000000018000669f     isfldsin003.exp
 0002:000026e7       $N00007                    00000001800066e7     isfldsin003.exp
 0002:00002727       $N00008                    0000000180006727     isfldsin003.exp
 0002:00002764       $N00009                    0000000180006764     isfldsin003.exp
 0002:0000279f       $N00010                    000000018000679f     isfldsin003.exp
 0002:000027cd       $N00011                    00000001800067cd     isfldsin003.exp
 0002:000027fe       $N00012                    00000001800067fe     isfldsin003.exp
 0002:0000282d       $N00013                    000000018000682d     isfldsin003.exp
 0002:0000285c       $N00014                    000000018000685c     isfldsin003.exp
 0002:00002891       $N00015                    0000000180006891     isfldsin003.exp
 0002:00002c9a       .idata$6                   0000000180006c9a     kernel32:KERNEL32.dll
 0002:00002cfe       .idata$6                   0000000180006cfe     vcruntime:VCRUNTIME140.dll
 0002:00002e6a       .idata$6                   0000000180006e6a     ucrt:api-ms-win-crt-runtime-l1-1-0.dll
 0002:00002e8c       .idata$6                   0000000180006e8c     ucrt:api-ms-win-crt-stdio-l1-1-0.dll
 0002:00002eac       .idata$6                   0000000180006eac     ucrt:api-ms-win-crt-string-l1-1-0.dll
 0003:00000000       ?codeAttributeName@@3PEBDEB 0000000180007000     libisfldsin003.obj
 0003:00000008       ?lineNumberAttributeName@@3PEBDEB 0000000180007008     libisfldsin003.obj
 0003:00000010       ?localVarAttributeName@@3PEBDEB 0000000180007010     libisfldsin003.obj
 0003:00000018       ?localVarTypeAttributeName@@3PEBDEB 0000000180007018     libisfldsin003.obj
 0003:00000020       ?stackMapAttributeName@@3PEBDEB 0000000180007020     libisfldsin003.obj
 0003:00000028       ?callBytes@@3PAEA          0000000180007028     libisfldsin003.obj
 0003:0000002c       ?allocBytes@@3PAEA         000000018000702c     libisfldsin003.obj
 0003:00000030       fields                     0000000180007030     libisfldsin003.obj
 0003:0001ab04       redefineAttempted          0000000180021b04     libisfldsin003.obj
 0003:0001ab08       nsk_context                0000000180021b08     libisfldsin003.obj
 0003:0001ab14       redefineSucceed            0000000180021b14     libisfldsin003.obj
 0003:0001ab18       agentFailed                0000000180021b18     libisfldsin003.obj
 0003:0001ab1c       currentAgentStatus         0000000180021b1c     libisfldsin003.obj
 0003:0001ab20       context                    0000000180021b20     libisfldsin003.obj
 0003:0001abd8       agentThread                0000000180021bd8     libisfldsin003.obj
 0003:0001abe0       agentThreadProc            0000000180021be0     libisfldsin003.obj
 0003:0001abe8       agentThreadArg             0000000180021be8     libisfldsin003.obj
 0003:0001abf0       agent_data                 0000000180021bf0     libisfldsin003.obj
 0003:0001ac00       jvmti_env                  0000000180021c00     libisfldsin003.obj
 0003:0001ac08       jvm                        0000000180021c08     libisfldsin003.obj
 0003:0001ac10       jni_env                    0000000180021c10     libisfldsin003.obj
 0003:0001ac18       checkStatus_func           0000000180021c18     libisfldsin003.obj
 0003:0001ac20       ?codeAttributeIndex@@3GA   0000000180021c20     libisfldsin003.obj
 0003:0001ac22       printdump                  0000000180021c22     libisfldsin003.obj
 0003:0001ac24       ?lineNumberAttributeIndex@@3GA 0000000180021c24     libisfldsin003.obj
 0003:0001ac28       ?localVarAttributeIndex@@3GA 0000000180021c28     libisfldsin003.obj
 0003:0001ac2c       ?localVarTypeAttributeIndex@@3GA 0000000180021c2c     libisfldsin003.obj
 0003:0001ac30       ?stackMapAttributeIndex@@3GA 0000000180021c30     libisfldsin003.obj
 0003:0001ac34       ?stackFrameOffset@@3GA     0000000180021c34     libisfldsin003.obj
 0003:0001ac38       ?mode@@3HA                 0000000180021c38     libisfldsin003.obj
 0003:0001ac3c       ?constantPoolSize@@3GA     0000000180021c3c     libisfldsin003.obj
 0003:0001ac40       ?orig@@3PEBEEB             0000000180021c40     libisfldsin003.obj
 0003:0001ac48       ?gen@@3PEAEEA              0000000180021c48     libisfldsin003.obj
 0003:0001ac50       ?inputPos@@3PEAEEA         0000000180021c50     libisfldsin003.obj
 0003:0001ac58       ?endPos@@3PEBEEB           0000000180021c58     libisfldsin003.obj
 0003:0001ac60       ?genPos@@3PEAEEA           0000000180021c60     libisfldsin003.obj
 0003:0001ac68       ?markPos@@3PEAEEA          0000000180021c68     libisfldsin003.obj
 0003:0001ac70       ?constantPool@@3PEAPEADEA  0000000180021c70     libisfldsin003.obj
 0003:0001ac78       ?constantPoolCount@@3GA    0000000180021c78     libisfldsin003.obj
 0003:0001ac7c       ?zeroBytes@@3PAEA          0000000180021c7c     libisfldsin003.obj
 0003:0001ac80       ?codeLength@@3IA           0000000180021c80     libisfldsin003.obj
 0003:0001ac84       result                     0000000180021c84     libisfldsin003.obj
 0003:0001ac88       ?map@@3PEAIEA              0000000180021c88     libisfldsin003.obj
 0003:0001ac90       ?widening@@3PEACEA         0000000180021c90     libisfldsin003.obj
 0003:0001ac98       jvmti                      0000000180021c98     libisfldsin003.obj
 0003:0001aca0       caps                       0000000180021ca0     libisfldsin003.obj
 0003:0001acc0       GS_ExceptionRecord         0000000180021cc0     MSVCRT:gs_report.obj
 0003:0001ad60       GS_ContextRecord           0000000180021d60     MSVCRT:gs_report.obj
 0003:0001b230       ?g_tss_cv@@3U_RTL_CONDITION_VARIABLE@@A 0000000180022230     MSVCRT:thread_safe_statics.obj
 0003:0001b238       ?g_tss_event@@3PEAXEA      0000000180022238     MSVCRT:thread_safe_statics.obj
 0003:0001b240       ?g_tss_mutex@@3U_RTL_CRITICAL_SECTION@@A 0000000180022240     MSVCRT:thread_safe_statics.obj
 0003:0001b268       ?g_sleep_condition_variable_cs@@3P6AHPEAU_RTL_CONDITION_VARIABLE@@PEAU_RTL_CRITICAL_SECTION@@K@ZEA 0000000180022268     MSVCRT:thread_safe_statics.obj
 0003:0001b270       ?g_wake_all_condition_variable@@3P6AXPEAU_RTL_CONDITION_VARIABLE@@@ZEA 0000000180022270     MSVCRT:thread_safe_statics.obj
 0003:0001b27c       ?__proc_attached@@3HA      000000018002227c     MSVCRT:dll_dllmain.obj
 0003:0001b290       ?is_initialized_as_dll@@3_NA 0000000180022290     MSVCRT:utility.obj
 0003:0001b291       ?module_local_atexit_table_initialized@@3_NA 0000000180022291     MSVCRT:utility.obj
 0003:0001b298       ?module_local_atexit_table@@3U_onexit_table_t@@A 0000000180022298     MSVCRT:utility.obj
 0003:0001b2b0       ?module_local_at_quick_exit_table@@3U_onexit_table_t@@A 00000001800222b0     MSVCRT:utility.obj
